:1000000012C0189518951895189518951895189563
:100010001895189518951895189518951895189578
:100020001895189518950FED0DBF00E002B903E380
:1000300009B906E003B900E00BB908E00AB905D038
:10004000000001E40CB90000FFCF0F930FB7F89444
:100050000F931F9308B30F9307B30F930FE34CD085
:1000600003EA4AD005EC48D006E946D00DE244D078
:100070000A2F42D00B2F40D00C2F3ED00D2F3CD05A
:1000800055D0C02F53D0D02F51D0A02F4FD0B02F4C
:100090004DD0003041F0013029F1023041F1033000
:1000A00059F0043099F00F9107BB0F9108BB1F91D5
:1000B0000F910FBF0F910895DFBBCEBBE09A0DB338
:1000C0000DB31AD021961197B9F7DACF2FD00DBB07
:1000D000DFBBCEBBE29AE19AE199FECF2196119760
:1000E000A9F7CECF099108D01197E1F7C9CF1ED05B
:1000F0000A931197E1F7C4CFBD9AC59A000000009A
:10010000000011E128D00894079551F018F0A89547
:10011000C59A03C0C598A895889411E11CD0F4CF66
:100120000000C5981FE118D0BD980895BD98A89506
:10013000B59BFDCF1FE110D00FE70000B59B02C0BB
:10014000889402C0089400000795A89511E103D097
:0E015000A0F30895000000001A95F1F708953D
:00000001FF
